:03004300021F0099
:03005300021F0089
:101F0000021E3400021E9100021E7B00021E4C00C5
:081F1000021C1F00021BA800C7
:101000001201000200000040AAAAAAAAAAAA01028C
:1010100003010A0600020000004001000902370037
:10102000020100C0000904000002FFFFFF040705E1
:101030000202000200070586020002000904010006
:1010400002FFFFFF050705040200020007058802F2
:10105000000200001201000200000040E4E451110F
:101060000000010203010A06000200000040010026
:1010700009023700020100C0320904000002FFFF2C
:10108000FF04070502024000000705860240000039
:101090000904010002FFFFFF0507050402400000EC
:1010A0000705880240000006040016001400120024
:1010B0000A00260004030904160358006F0072009A
:1010C00063006F006D0020004C00540044001403C6
:1010D00041007300740072006900620061006E00DC
:1010E0006B001203530065007200690061006C0020
:1010F0004E006F000A0346005000470041002603DF
:101100004D0061006E00610067006D0065006E00BB
:101110007400500072006F0063006500730073007C
:061120006F0072000000E8
:051EF1000300000000E9
:1011F50041E0370041E0B70042E0B2000041E0388D
:1012050000021BE0860218E07A43E0B40000004EBD
:10121500E03931313435314D502020202020200057
:101D9A008B518A528953E5561556AE557002155520
:101DAA004E6014AB510553E553AA52700205521402
:081DBA00F9ED12077180DF2230
:101BE5008B518A528953E5581558AE5770021557CF
:101BF5004E6026AB540556E556AA55700205551498
:101C0500F912072BFFAB510553E553AA5270020594
:0A1C15005214F9EF12077180CD227E
:101D7000C2B5C2B7E490E670F075B5E653B5EE4370
:101D8000B28053B2F4A2B53390E0B7F0C2B3C2B69A
:0A1D90007F327E00121E0AD2B62236
:101E6400538EF75389FB5389F74389015389FDE462
:071E7400F58AF58CD2A922CA
:1017B7008C428D43AA06A9077554018A5589567527
:1017C700570075581C7B017AE0794D121BE590E0B4
:1017D7004DE0B4C20374C0F090E065E0FCA3E0FD07
:1017E700A3E0FEA3E064D1FFEE648DFEED644CFD43
:1017F700EC6449FC90E06512084D7EE07F4D7D1C4E
:101807007C001213647EE07F4D7B1C7A00AD43ACF5
:10181700421214187D1C7C00AF43AE42120F367D76
:0A1827001C7C00AF43AE42021C55CA
:0818A9008E428F438C448D45F3
:1018B100C20712001290E15CEFF0BF5004D2078022
:1018C10057E490E15DF0A3F090E15DE0FEA3E0FF5D
:1018D100C39410EE648094805030E5452FF582E585
:1018E100443EF583E0FF90E15DE0FCA3E02543F594
:1018F10082E5423CF583E0B5071090E15EE004F03B
:1019010070C690E15DE004F080BE90E15DE070049E
:0A191100A3E064107002D207A207E1
:01191B0022A9
:020E0C008F3F16
:100E0E001200128F40E4F544F545AD45AC44121482
:100E1E00CE746A2545F582E434E0F583E541F005AC
:100E2E0045E54570020544C39408E544648094800A
:100E3E0040D8E53F600490E06AF090E06AE0B4C00C
:100E4E0008754200754308800675421D7543367558
:100E5E004400754508C3E5459410E54464809480CC
:100E6E0050231214CA746A2545F582E434E0F583E2
:100E7E00E541F00545E545700205440543E543703F
:100E8E00D4054280D07541FF75421D7543197544D6
:100E9E0000754510C3E545942CE54464809480505C
:100EAE0033E540B4510E7B007A007941AD43AC423C
:100EBE00FF1214D6746A2545F582E434E0F583E515
:100ECE0041F00545E545700205440543E54370C410
:100EDE00054280C075421D75433EE4F541F544F56B
:100EEE0045C3E5459406E54464809480502FE54063
:100EFE00B4510A90E06AE0B4C2031214CA744725D2
:100F0E0045F582E434E0F583E541F00545E54570AD
:100F1E000205440543E54370C8054280C490E06A6B
:070F2E00E0B4C20374C0F03F
:010F35002299
:0A1982008E428F438B448A4589464C
:10198C007E00E5432DF54BEE3542F54A1200128FE1
:10199C0047E5476451600BC3E5439410E54294005E
:1019AC005035854248854349C3E549954BE54895F3
:1019BC004A5024AB44AA45A946AD49AC48AF47129E
:1019CC0017340549E5497002054874012546F5466A
:0719DC00E43545F54580D11B
:0119E30022E1
:061831008B3F8A40894153
:10183700D2067554017555E075566A755700755887
:10184700107B017AE07996121BE5E5412410F9E453
:101857003540853F54F555895675570075580C7BAB
:10186700017AE079A6121BE57EE07F967CE07D1A7F
:101877001217B77EE07F1AE541241CF9E43540FCD6
:10188700AD011218A95016AB3FE5412410F9E43514
:1018970040FA7D1C7F197E1D1219828002C206A2A2
:0118A700063A
:0118A800221D
:101126007F03121D45EF2402FFE43EA907753F0128
:10113600F540894190E06BE0FFE50C2408F582E478
:10114600350BF583EFF090E06CE0FFE50C2409F534
:1011560082E4350BF583EFF090E06DE0FFE50C24BB
:101166000AF582E4350BF583EFF090E06EE0FFE5DB
:101176000C240BF582E4350BF583EFF090E06FE07D
:10118600FFE50C240CF582E4350BF583EFF090E0D7
:1011960070E0FFE50C240DF582E4350BF583EFF0E6
:1011A6007F087E00E4FDEDC394085028746A2FF58D
:1011B60082E434E0F583E0FCAB3FAA40A94175F038
:1011C60002EDA4F58285F083EC1207830D0FBF00B4
:1011D600010E80D2E5192404F582E43518F583E082
:0E11E60030E0047F0180027F0090E037EFF0E0
:0111F40022D8
:101B240090E06DE02FFFE50C240AF582E4350BF517
:101B340083EFF0E50C240BF582E4350BF583E0FE2E
:101B4400E50C240AF582E4350BF583E0FDEDFF9006
:101B5400E0B2EEF0A3EFF0D206121CBC90E680E0F7
:041B640054F7F02220
:1016140090E600E054E74410F090E60174C0F090C6
:10162400E6107420F000000090E611F00000009035
:10163400E6047480F0000000740FF0000000E4F091
:1016440000000090E6187410F0000000E490E61921
:10165400F000000090E61A7408F0000000E490E640
:101664001BF000000090E6497482F0000000F000D6
:10167400000090E6247402F0000000E490E625F0F7
:1016840000000090E6957480F0000000F000000077
:1016940043AF017B017AE07914755500755606E471
:0416A400FD021D9A8C
:061E0400D2877F0A7E0078
:101E0A007C007D181207A5EF1FAC0670011E4C70EE
:021E1A00F622AE
:0A1A3D008E3F8F408B418A4289439F
:101A4700E4F544F545C3E5459540E544953F503BEE
:101A5700AB41AA42A943854582854483120744FFC7
:101A6700E4FBFAC2B2EF1392B7EFC313FFD2B20B84
:101A7700BB00010AEB64084A70E9C2B220B002C396
:0C1A8700220545E54570BE054480BAD339
:011A93002230
:101E1C0090E60174C0F0C2B67F967E00121E0AD204
:081E2C00B67F327E00021E0A9F
:101EA700D2B1121E04C2B1121E06C2877F0A7E007B
:031EB700021E0AFE
:021B6800AB07C9
:101B6A00E4F9FAEBC413131354011392B17F027E02
:101B7A0000121E0AD2877F057E00121E0AE925E09E
:101B8A00FFA283E4334FF97F057E00121E0AEB257C
:0D1B9A00E0FBC287121E060ABA08C8AF01A0
:011BA700221B
:061A94008B538A548955B2
:101A9A00A2AFE433F55B121EA7E4F55AE55AC395E3
:101AAA00595027AB53AA54A955855A8275830012F7
:101ABA000744FF121B68AB56AA57A958855A827564
:101ACA008300EF120783055A80D2120036E55B24A1
:031ADA00FF92AFC9
:011ADD0022E6
:0B003600C2B1121E06121E04D2B1223D
:101DEA00753F8F8F4075560075570075584975595C
:0A1DFA00027B007A00793F021A9480
:101C8B00783F7C007D007BFF7A1E79F17E007F051B
:101C9B0012070530B41575560075570075583F750A
:101CAB0059057B007A00793F121A94E5415401FFE4
:011CBB002206
:100B4800753F007540007541007543017544E075B7
:100B580045007546017547E0754808E4F54FFFF50F
:100B6800507B017AE07900F555755608FD121D9AFB
:100B7800AB43AA44A9457401120771E4F54EE54E4A
:100B8800C454F0AB43AA44A94590000112078385D9
:100B98004656854757854858755908121A94AB46E2
:100BA800AA47A948900002120744FE5407FFEE54D2
:100BB80070F54F24E0602924F0604B24F0605D2438
:100BC800F0606F24406003020C50753F01851840A7
:100BD800851941EF24FE600624FE703B801C801FAF
:100BE800E5192401FDE43518A905753F01F540898B
:100BF80041EF24FC60092402700A75500280527586
:100C08005006804D8011E5192402FDE43518A90528
:100C1800753F01F54089417550088035E519240371
:100C2800FDE43518A905753F01F540894175500463
:100C3800801FE5192405FDE43518A905753F01F560
:100C48004089417550988009753F0075400075418D
:100C580000E5404541453F6022AB3FAA40A941120B
:100C6800072BFED395504006AD50AE0580008E424E
:100C780012072BC39542120771800CE54F70047E52
:100C88000180027E008E427449254EF8A642054E28
:100C9800E54EC394055003020B86AB43AA44A9450D
:100CA8007488120771AB43E5452401F9E43544FA29
:100CB80075540075550075564975570075580512D5
:100CC8001BE5854656854757854858755908AB43EF
:070CD800AA44A945021A9489
:1019E4008F3F90E0B2E0FEA3E054F064607003EE39
:1019F400641160037F012290E037E070037F0F22BF
:101A0400E53F7003308108E53FB401062080037F81
:101A1400102290E0B7E0B53F037F0122E4F511D234
:101A240006121CBCAF3F90E0B7EFF024FF92B590D4
:091A3400E680E054F7F07F002287
:04000E0090FC04F06E
:1000120090E678E0541824F06008240870087F50B5
:0800220080067F518002E4FF1B
:01002A0022B3
:0C14CA00AD43AC427B007A007941AF409A
:0C14D6008F468C478D488B498A4A894B11
:1014E200E4F54CF54D754E03FDF54FF550A2AF33C3
:1014F200F551E54624AF600D047012754C00754D30
:10150200017D018008754C00754D02E4FDE54660E1
:1015120051E54D454C604BE54790E0B4F0E548A3FA
:10152200F074B42DF582E434E0AD82FCAB4DAF46ED
:1015320012191C754F008F507F0A7E00121ADEE5C9
:1015420050454F60107CE07D697B01AF4612156FFC
:10155200754F008F5090E069E0AB49AA4AA94B123F
:0C1562000771E55124FF92AFAE4FAF506F
:01156E00225A
:0C1734008F4C8C4D8D4E8B4F8A5089518C
:10174000E4F552F553755403FDF555F556A2AF3344
:10175000F557E54C24AF600D0470127552007553B7
:10176000027D018008755200755303E4FDE54C606D
:101770003BE55345526035E54D90E0B4F0E54EA3AE
:10178000F0AB4FAA50A95112072B90E0B6F074B4F9
:101790002DF582E434E0AD82FCAB53AF4C12191C42
:1017A0007555008F567F0A7E00121ADEE55724FF1A
:0617B00092AFAE55AF56EA
:0117B6002210
:10005600E4F531F532F535F53AF53BF53CF53DE598
:10006600AA5484600302063490E694E0FE90E69576
:10007600E0FBEEF53AEBF53BC39405E53A94004018
:100086000790F404E0FD80027DFFED12085900CED2
:100096000102B905030007035F0903C80B011E0E21
:1000A60000E40F01941102541305312503F13104C4
:1000B6004732045A3404A23504B93604D63703D578
:1000C6004503E647000005B475310075320790FC1C
:1000D600047481F0A37414F0E4A3F00205D77F0F33
:1000E600121DEA75310075320690FC047480F0E446
:1000F600A3F0753505F511FE74002535F9EE34F4D7
:10010600FA7B01121831400690FC05740EF0E4FFEC
:10011600120E0C7F8F0202B37F0E121DEA7531009C
:10012600753205748E12000E8F3D7B007A00793E83
:10013600E4FDFC1214D6E53D64516019E53D6450BA
:10014600601375310075320690FC047480F0A37458
:100156000BF00205D790E0B8E0FF120E0C740025F4
:1001660032F974FC3531FA7B01C0038B547555E0C6
:1001760075566A75570075582CD003121BE5742CFA
:100186002532F532E43531F5317F8E0202B3753111
:100196000075320790FC047491F090E678E090FCCC
:1001A60005F030B4047F0180027F0090FC06EFF07A
:1001B60074002532F974FC3531FA7B0175550075EA
:1001C6005612E4FD121D9A74002532F974FC35317D
:1001D600FA7B01C0038B547555E075563975570087
:1001E600755806D003121BE574062532F532E43540
:1001F60031F531FE74002532F974FC3EFA7B01C0FC
:10020600038B547555E0755614755700755806D00E
:1002160003121BE574062532F532E43531F531FE5D
:1002260074002532F974FC3EFA7B01C0038B5475C9
:1002360055E0755647755700755806D003121BE5ED
:1002460074062532F532E43531F5310205D77F13D0
:10025600121DEA75310075321D749312000E8F3D22
:1002660075381D753900753600753705D3E539942F
:1002760018E538941D5034E53DB4510E7B007A00E4
:10028600793EAD39AC38FF1214D674002537F582A5
:1002960074FC3536F583E53EF00539E5397002051F
:1002A600380537E53770C5053680C17F93121DEADC
:1002B6000205D775310075320690FC047480F0E4AF
:1002C600A3F090F405E090E038F0E014702A30B026
:1002D6001E121E1C7554017555F475560675570089
:1002E6007558067B017AE07914121BE50205D79052
:1002F600FC057401F00203C08056753100753206A4
:1003060090FC047480F0E4A3F0753507AF35FEC3A6
:10031600E53B9FF534E53A9EF53390E038E01470FE
:100326002F20B00330B42074002FF974F43EFA7B0A
:1003360001AF34AE33121A3D5004E40204B290FC0D
:1003460005740CF00205D790FC057402F00205D77F
:1003560090FC057403F00205D775310075320690DE
:10036600FC047480F0E4A3F090E038E014704530AB
:10037600B43A90E6017403F07F647E00121E0A9080
:10038600E0B8E0FF120E0C7EE07F6A7CE07DB912D9
:1003960017B77EE07FB9AD1CAC1B1218A950051229
:1003A6000B48801690FC05740EF0800E90FC0574C8
:1003B6000DF0800690FC057403F0E490E038F0023E
:1003C60005D7E4F531F5327F02121B240205D7E486
:1003D600FF120E0C121126E4FF1219E4E4FF80024C
:1003E6007F01121B24121E1C0205D77531007532BF
:1003F6000690FC047480F0E4A3F090F405E0F53C6C
:10040600E4F511E53C64016004E53C703290E0B22D
:10041600E0FEA3E054F064607003EE6411600280B5
:100426007290E037E070028058E5116401600AE5D9
:1004360011700C121C8BEF6006853C110205D780EB
:100446005275310075320690FC0474B2F0A3E511C2
:10045600F00205D775310075320690FC047480F001
:10046600E4A3F090F405E0F53CFF1219E4EF24F163
:10047600600F1460152410701AE4F531F532020588
:10048600D790FC05740FF00205D790FC057410F0A8
:100496000205D790FC057401F00205D77531007589
:1004A600320690FC0474B5F090E0B7E090FC05F0DD
:1004B6000205D775310075320690FC0474B6F0A2B9
:1004C60080E43325E0FFA281E4334FA3F00205D791
:1004D600853A31853B3290FC0474B7F0753505C317
:1004E600E53B9535F534E53A9400F533740025354A
:1004F600F582E434F4F583E0648870030205D7AF2F
:10050600357E0074002FF9EE34F4FA7B01C003C087
:100516000174002FF9EE34FC8B56F5578958853453
:1005260059D001D003121A940205D77531007532DD
:100536000590FC0474A5F01200128F3D7B007A0032
:10054600793EE4FDFC1214D690E036E0FF0532E574
:1005560032AC3170020531142400F58274FC3CF58E
:1005660083EFF090E0B8E0FF0532E532AC3170027F
:100576000531142400F58274FC3CF583EFF0053256
:10058600E532AE3170020531142400F58274FC3E6A
:10059600F583E53EF00532E532AE317002053114E1
:1005A6002400F58274FC3EF58374FFF080237531D8
:1005B6000075320690FC047480F0C3E53B9405E5B3
:1005C6003A94005006A37407F0800690FC05740662
:1005D600F090F404E0B48004A3E0701290F404E018
:1005E6006405600FE06407600AE064096005E49052
:1005F600E038F0E5324531602CE532FD90FC00F044
:10060600E531FFA3F090F402E090FC02F090F403D1
:10061600E090FC03F090E69CEFF000000090E69D71
:0E062600EDF000000090E6957480F0000000FA
:0106340022A3
:02004100D322C8
:0800030090E6BAE0F51DD322DE
:101ECD0090E740E51DF0E490E68AF090E68B04F093
:021EDD00D3220E
:08002B0090E6BAE0F51AD322B9
:101EDF0090E740E51AF0E490E68AF090E68B04F084
:021EEF00D322FC
:101DC20090E6B9E0242F600D04701990E604E0FF5C
:101DD200430780800890E604E0FF53077F0000007D
:071DE200EFF08002D322C3E1
:011DE90022D7
:101E3400C0E0C083C082D2015391EF90E65D74018B
:081E4400F0D082D083D0E0321F
:101E7B00C0E0C083C0825391EF90E65D7404F0D054
:061E8B0082D083D0E0329A
:101E9100C0E0C083C0825391EF90E65D7402F0D040
:061EA10082D083D0E03284
:101C1F00C0E0C083C08285120D85130E850E8285AC
:101C2F000D83A37402F085090F850A108510828534
:101C3F000F83A37407F05391EF90E65D7410F0D00B
:061C4F0082D083D0E032D8
:101E4C00C0E0C083C082D2035391EF90E65D74086A
:081E5C00F0D082D083D0E03207
:101BA800C0E0C083C08290E680E030E72085090D60
:101BB800850A0E850E82850D83A37402F085120FA7
:101BC800851310851082850F83A37407F05391EF56
:0D1BD80090E65D7420F0D082D083D0E03222
:101EBA00000102020303040405050300000000C038
:031ECA00C2000053
:06122500011100010800A8
:03000B000212B02E
:1012B000C0E0C0F0C083C082C0D075D000C000C004
:0D12C00001C002C003C004C005C006C00785
:1012CD0078217C007D007BFF7A1E79C47E007F052E
:1012DD0012070590E0B7E0F526C204752700E50872
:1012ED00600415088056750805E5117004C2048068
:1012FD0043A280308101B3500B3081047F008030D8
:10130D007F01802C30B41575560075570075582126
:10131D007559057B007A007921121A94E523540141
:10132D00F527701090E0B7E060047F0080027F0128
:0C133D008F26D204300405AF261219E4FC
:10134900D007D006D005D004D003D002D001D000F8
:0B135900D0D0D082D083D0F0D0E032A2
:100CDF0078577CE17D017BFF7A1E79C97E007F0406
:100CEF00120705C203C200D202C201121D70121EEA
:100CFF0064121614750B10750C00751410751512FF
:100D0F00750910750A1C75121075137085120F85F1
:100D1F0013107516107517B412001290E155EFF0FD
:100D2F007B017AE17956E4FDFC1214D690E156E08E
:100D3F00FF90E036F0E490E0B8F0EF64C26059EF56
:100D4F0064C06054E490E15BF090E15BE0FFC3941A
:100D5F0004504A74572FF582E434E1F583E0FF60C5
:100D6F003C120E0C7EE07F6A7CE07DB91217B77ED5
:100D7F00E07FB9AD1CAC1B1218A9501490E15BE0D9
:100D8F002457F582E434E1F583E090E0B8F0800D6C
:100D9F0090E15BE004F080B1E4FF120E0C1211261B
:100DAF00D2E843D82090E668E04409F090E65CE092
:100DBF00443DF012001290E155EFF07B017AE1799A
:100DCF0056E4FDFC1214D690E156E064C26007E4CD
:100DDF0090E0B7F0C2B57F01121B24D2AFD28C5373
:100DEF008EF8C203C2AF120056D2AF3001051209FE
:0D0DFF0020C2013003EEC203121D1980E76F
:0B00460090E50DE030E402C322D3225D
:1009200090E6B9E070030209E5147003020A5A2444
:10093000FE7003020AD524FB70030209DF14700362
:100940000209D91470030209CD1470030209D324DB
:10095000056003020B341200414003020B4090E695
:10096000BBE024FE602714603E24FD601114602764
:1009700024067056E50B90E6B3F0E50C80421200B9
:10098000465044E51490E6B3F0E5158033E50D904C
:10099000E6B3F0E50E802985120F851310E50F9060
:1009A000E6B3F0E510801990E6BAE0FF121D45AA03
:1009B00006A9077B01EA494B600DEE90E6B3F0EF24
:1009C00090E6B4F0020B40020B2F020B2F121EDF39
:1009D000020B4012002B020B40120003020B4012CC
:1009E0001ECD020B4090E6B8E0247F60151460191C
:1009F00024027063A200E43325E0FFA202E4334F37
:100A00008041E490E740F0803F90E6BCE0547EFFF8
:100A10007E00E0D394807C0040047D0180027D0054
:100A2000EC4EFEED4F24BAF582741E3EF583E4933E
:100A3000FF3395E0FEEF24A1FFEE34E68F82F583CD
:100A4000E0540190E740F0E4A3F090E68AF090E6ED
:100A50008B7402F0020B40020B2F90E6B8E024FEEC
:100A6000601624026003020B4090E6BAE0B4010570
:100A7000C200020B40020B2F90E6BAE0705590E6E0
:100A8000BCE0547EFF7E00E0D394807C0040047D77
:100A90000180027D00EC4EFEED4F24BAF582741EFB
:100AA0003EF583E493FF3395E0FEEF24A1FFEE349F
:100AB000E68F82F583E054FEF090E6BCE0548013AC
:100AC0001313541FFFE0540F2F90E683F0E04420EF
:100AD000F0806D805A90E6B8E024FE601924027020
:100AE0004E90E6BAE0B40104D200805490E6BAE039
:100AF0006402604C803990E6BCE0547EFF7E00E0EA
:100B0000D394807C0040047D0180027D00EC4EFE89
:100B1000ED4F24BAF582741E3EF583E493FF3395BE
:100B2000E0FEEF24A1FFEE34E68F82F583800D9086
:100B3000E6A08008121DC2500790E6A0E04401F034
:070B400090E6A0E04480F004
:010B4700228B
:03003300021EF6B4
:041EF60053D8EF329C
:10122B006080E0D5292E43C9A2D87C013D3654A15C
:10123B00ECF0061362A705F3C0C7738C98932BD9F8
:10124B00BC4C82CA1E9B573CFDD4E01667426F18FC
:10125B008A17E512BE4EC4D6DA9EDE49A0FBF58E88
:10126B00BB2FEE7AA968799115B2073F94C210890A
:10127B000B225F21807F5D9A5A903227353ECCE757
:10128B00BFF79703FF1930B348A5B5D1D75E922AA4
:10129B00AC56AAC64FB838D296A47DB676FC6BE294
:0412AB009C7404F13A
:081364008C448D45AB07AA067D
:10136C00E4F546F547C3E5479545E5446480F8E563
:10137C00466480984003021413E54725E0FFE546D8
:10138C0033FE74D52FF58274E03EF583E0FF7E00CA
:10139C00AC44AD451207B78C488D49E54725E0FFB5
:1013AC00E54633FE74D62FF58274E03EF583E0FFFC
:1013BC007E00AC44AD451207B78C4A8D4BE54965B0
:1013CC004B7004E548654A6030EB2549F582EA35F7
:1013DC0048F583E0F9EB254BF582EA354AF583E0D5
:1013EC00FFEB2549F582EA3548F583EFF0EB254B09
:1013FC00F582EA354AF583E9F00547E547600302D3
:0B140C00137105460213717E007F0182
:0114170022B2
:0C1418008E448F458C468D478A488B49D6
:10142400E54545446006E54745467004E4FEFF2271
:10143400E4F54AF54BC3E54B9549E5486480F8E586
:101444004A648098507BE4F54CF54DE547254BF50F
:1014540082E546354AF583E4F0C3E54D9549E54810
:101464006480F8E54C6480985049E54D254B24D5BB
:10147400F582E434E0F583E0FFE545254DF582E5AA
:1014840044354CF583E0FEEF8EF0A4FFE547254B91
:10149400F582E546354AF583E02FFFE547254BF510
:1014A40082E546354AF583EFF0054DE54D70AA0512
:1014B4004C80A6054BE54B6003021439054A02141F
:0514C400397E007F01EC
:0114C9002200
:101CEB0012072BFF90000312074412077190000399
:101CFB00EF120783900002120744FF9000011207B6
:0E1D0B0044900002120783900001EF0207834C
:080F36008E448F458C468D4767
:100F3E00E4F548F549E547AE467802CEA2E713CE72
:100F4E0013D8F8FFC3E5499FEE6480F8E548648046
:100F5E00984003020FF8E549AE487802C333CE330A
:100F6E00CED8F92545FFEE3544FAA9077B018B4A09
:100F7E00F54B894C74D62549F582E434E0F583E0CF
:100F8E00541FFFE48F50F54FF54EF54D121CEBAB91
:100F9E004AAA4BA94C120813C374209550F9F812A3
:100FAE000800C004C005C006C007A94C120813A94A
:100FBE0050A8011207EDD003D002D001D000EF4BA4
:100FCE00FFEE4AFEED49FDEC48FCAB4AAA4BA94C9C
:100FDE00120833AB4AAA4BA94C121CEB0549E54942
:0E0FEE006003020F430548020F437E007F019F
:010FFC0022D2
:101C5500D3ED9410EC64809480402AED1D70011C36
:101C6500142FF582EE3CF583E0FB547F24D5F582F5
:101C7500E434E0F583E0F9540F2FF582E43EF58373
:051C8500E06BF080CBD4
:011C8A002237
:101D190090E682E030E004E020E60B90E682E030D5
:101D2900E119E030E71590E680E04401F07F147E88
:0C1D390000121ADE90E680E054FEF0225A
:101CBC0030060990E680E0440AF0800790E680E068
:101CCC004408F07FDC7E05121ADE90E65D74FFF0AE
:0F1CDC0090E65FF05391EF90E680E054F7F0222E
:101ADE008E588F5990E600E054187012E559240183
:101AEE00FFE43558C313F558EF13F559801590E6FA
:101AFE0000E05418FFBF100BE55925E0F559E558E5
:101B0E0033F558E5591559AE58700215584E600503
:061B1E00121F1880EE22E8
:06156F008C528D53AE0703
:10157500EB70037F012290E678E020E6F990E678AB
:101585007480F0EE25E0440190E679F090E678E08D
:1015950030E0F990E678E020E26BE030E167BB01EE
:1015A5000790E678E04420F090E679E0F5541BEBEF
:1015B500603090E678E030E0F990E678E020E245AA
:1015C500BB010790E678E04420F090E679E0FF055E
:1015D50053E553AC527002055214F5828C83EFF03B
:1015E50080CC90E678E030E0F990E678E020E215EE
:1015F50090E678E04440F090E679E08553828552A4
:0E16050083F07F012290E678E04440F07F0001
:0116130022B4
:10191C0090E678E020E6F990E6787480F0EF25E028
:10192C0090E679F090E678E030E0F990E678E02007
:10193C00E23AE030E136EBD3940040260DEDAE04F4
:10194C0070010C14F5828E83E090E679F01B90E622
:10195C0078E030E0F990E678E020E210E020E1D683
:10196C00800A90E678E04440F07F012290E678E02F
:05197C004440F07F0073
:011981002243
:021D4500A907EC
:101D4700AE16AF178F828E83A3E064037017AD01C1
:101D570019ED7001228F828E83E07C002FFDEC3E0F
:081D6700FEAF0580DFE4FEFF82
:011D6F002251
:101F18007400F58690FDA57C05A3E582458370F9DC
:011F28002296
:030000000216A83D
:0C16A800787FE4F6D8FD75815B0216EF38
:10063500E709F608DFFA8046E709F208DFFA803EA7
:1006450088828C83E709F0A3DFFA8032E309F60894
:10065500DFFA8078E309F208DFFA807088828C83FC
:10066500E309F0A3DFFA806489828A83E0A3F608B0
:10067500DFFA805889828A83E0A3F208DFFA804C8A
:1006850080D280FA80C680D4806980F28033801061
:1006950080A680EA809A80A880DA80E280CA8033CA
:1006A50089828A83ECFAE493A3C8C582C8CCC58342
:1006B500CCF0A3C8C582C8CCC583CCDFE9DEE78012
:1006C5000D89828A83E493A3F608DFF9ECFAA9F091
:1006D500EDFB2289828A83ECFAE0A3C8C582C8CCE7
:1006E500C583CCF0A3C8C582C8CCC583CCDFEADE00
:1006F500E880DB89828A83E493A3F208DFF980CC62
:1007050088F0EF60010E4E60C388F0ED2402B4045A
:100715000050B9F582EB2402B4040050AF23234501
:060725008223900685739B
:10072B00BB010689828A83E0225002E722BBFE02CC
:09073B00E32289828A83E49322FF
:10074400BB010CE58229F582E5833AF583E022506A
:1007540006E92582F8E622BBFE06E92582F8E222B4
:0D076400E58229F582E5833AF583E49322CE
:10077100BB010689828A83F0225002F722BBFE0167
:02078100F32261
:10078300F8BB010DE58229F582E5833AF583E8F0AC
:10079300225006E92582C8F622BBFE05E92582C858
:0207A300F22240
:1007A500EF8DF0A4A8F0CF8CF0A428CE8DF0A42E68
:0207B500FE2222
:1007B700C2D5EC30E709B2D5E4C39DFDE49CFCEE5D
:1007C70030E715B2D5E4C39FFFE49EFE12087FC34E
:1007D700E49DFDE49CFC800312087F30D507C3E449
:0607E7009FFFE49EFE22CC
:1007ED00E8600FECC313FCED13FDEE13FEEF13FFEA
:0307FD00D8F1220E
:10080000E8600FEFC333FFEE33FEED33FDEC33FC56
:03081000D8F122FA
:10081300BB010789828A830208E05005E9F80208D0
:10082300D4BBFE05E9F80208EC89828A830208F842
:10083300BB010789828A8302084D5005E9F8020942
:0A08430008BBFE05E9F802091422C3
:0C084D00ECF0A3EDF0A3EEF0A3EFF0221E
:10085900D083D082F8E4937012740193700DA3A32E
:1008690093F8740193F5828883E473740293686042
:06087900EFA3A3A380DF42
:1016B400020CDFE493A3F8E493A34003F68001F261
:1016C40008DFF48029E493A3F85407240CC8C33337
:1016D400C4540F4420C8834004F456800146F6DF06
:1016E400E4800B01020408102040809011F5E47E90
:1016F400019360BCA3FF543F30E509541FFEE493FB
:10170400A360010ECF54C025E060A840B8E493A3C1
:10171400FAE493A3F8E493A3C8C582C8CAC583CAEC
:10172400F0A3C8C582C8CAC583CADFE9DEE780BEA4
:0112AF00003E
:10087F00BC000BBE0029EF8DF084FFADF022E4CC5D
:10088F00F875F008EF2FFFEE33FEEC33FCEE9DEC26
:10089F00984005FCEE9DFE0FD5F0E9E4CEFD22ED6C
:1008AF00F8F5F0EE8420D21CFEADF075F008EF2FB6
:1008BF00FFED33FD4007985006D5F0F222C398FDA7
:0508CF000FD5F0EA2244
:0C08D400E6FC08E6FD08E6FE08E6FF2250
:0C08E000E0FCA3E0FDA3E0FEA3E0FF228B
:0C08EC00E2FC08E2FD08E2FE08E2FF2248
:1008F800E493FC740193FD740293FE740393FF2246
:0C090800ECF608EDF608EEF608EFF6221B
:0C091400ECF208EDF208EEF208EFF2221F
:00000001FF
